:0200000480007A
:100000006F00C004732F2034930F8000630AFF0336
:10001000930F90006306FF03930FB0006302FF038A
:10002000170F0080130F0FFE63040F0067000F000F
:10003000732F203463540F006F004000136E9E53E3
:10004000171F00002320CFFD6FF09FFF732540F1A5
:100050006310050073251030635805000F00F00F82
:10006000130E100073000000130E00009702000032
:10007000938282F973905230735020307350303035
:1000800073504030970200809382C2F7638C020065
:10009000739052109302B01A739022307323203061
:1000A000E39E62F873500030970200009382420191
:1000B00073901234732540F173002030130E20002A
:1000C0009300000013010000638620006318C02B1A
:1000D0006316C001E38E20FE6312C02B130E3000A6
:1000E0009300100013011000638620006318C029DC
:1000F0006316C001E38E20FE6312C029130E400078
:100100009300F0FF1301F0FF638620006318C027FF
:100110006316C001E38E20FE6312C027130E500049
:100120009300000013011000638420006314C001D9
:100130006316C025E38E20FE130E600093001000AE
:1001400013010000638420006314C0016318C023FE
:10015000E38E20FE130E70009300F0FF13011000D9
:10016000638420006314C001631AC021E38E20FE63
:10017000130E8000930010001301F0FF6384200031
:100180006314C001631CC01FE38E20FE130E900099
:1001900013020000930000001301F0FF6380201E93
:1001A0001302120093022000E31652FE130EA00069
:1001B00013020000930000001301F0FF1300000081
:1001C000638E201A1302120093022000E31452FEE1
:1001D000130EB00013020000930000001301F0FFA3
:1001E0001300000013000000638A2018130212009D
:1001F00093022000E31252FE130EC000130200000F
:1002000093000000130000001301F0FF6388201624
:100210001302120093022000E31452FE130ED000CA
:100220001302000093000000130000001301F0FF10
:1002300013000000638420141302120093022000B4
:10024000E31252FE130EE0001302000093000000C0
:1002500013000000130000001301F0FF6380201260
:100260001302120093022000E31252FE130EF0005C
:1002700013020000930000001301F0FF63802010C0
:100280001302120093022000E31652FE130E000127
:1002900013020000930000001301F0FF13000000A0
:1002A000638E200C1302120093022000E31452FE0E
:1002B000130E100113020000930000001301F0FF61
:1002C0001300000013000000638A200A13021200CA
:1002D00093022000E31252FE130E200113020000CD
:1002E00093000000130000001301F0FF6388200852
:1002F0001302120093022000E31452FE130E300189
:100300001302000093000000130000001301F0FF2F
:1003100013000000638420061302120093022000E1
:10032000E31252FE130E400113020000930000007E
:1003300013000000130000001301F0FF638020048D
:100340001302120093022000E31252FE93001000E9
:10035000630A0000938010009380100093801000C7
:10036000938010009380100093801000930E300053
:10037000130E50016394D001631CC0010F00F00FF5
:1003800063000E00131E1E00136E1E00730000009B
:100390000F00F00F130E100073000000731000C068
:1003A000000000000000000000000000000000004D
:1003B000000000000000000000000000000000003D
:0403C0000000000039
:1010000000000000000000000000000000000000E0
:1010100000000000000000000000000000000000D0
:1010200000000000000000000000000000000000C0
:1010300000000000000000000000000000000000B0
:081040000000000000000000A8
:040000058000200057
:00000001FF
